:020000040000FA
:020000002FD1FE
:06000800FACF0BF072D0EC
:080018000E6ED8CF0FF0E0CF0F
:100020000DF0FACF0CF08A6A896AFF0E926E896E23
:100030003C2A400E3C6402D0010E3C6E406A3C50AB
:100040003D6040843E6040823F6040808B50F80BB2
:10005000401009B0070A8B6E0DEC01F0F9501450F6
:10006000F92638D030D028D020D018D010D008D0E1
:100070002C1C926E146A800E8A6EB6EC00F030D0A2
:100080002B1C926E0E0E146E400E8A6E29D02A1C06
:10009000926E0C0E146E200E8A6E22D0291C926E67
:1000A0000A0E146E100E8A6E1BD0281C926E080E5B
:1000B000146E080E8A6E14D0271C926E060E146EF3
:1000C000040E8A6E0DD0261C926E040E146E020E63
:1000D0008A6E06D0251C926E020E146E010E8A6E78
:1000E000F2940DC0E0FF0E500FC0D8FF0CC0FAFF15
:1000F00010009E92337033B036D034663406C1ECB3
:100100000DF0E86620D055A41ED0525002620CD0EB
:100110005150036209D00830010B316E010E0814F2
:10012000311802E1559E0FD0525004620CD051504C
:10013000056209D00830E830010B316E010E081459
:10014000311801E1558E594E07D0020E59620BD07D
:100150008250300B586E07D0030E596E8250300B10
:10016000586201D0576E0BC0FAFF1100396611D0EA
:1001700015C025F016C026F017C027F018C028F0CB
:1001800019C029F01AC02AF01BC02BF01CC02CF09B
:100190001200382E08D037C038F03B2E04D039C0BA
:1001A0003BF03A2C3A6E3A50385CD8B0E1D71DC0DB
:1001B00025F01EC026F01FC027F020C028F021C067
:1001C00029F022C02AF023C02BF024C02CF012000A
:1001D00015C01DF016C01EF017C01FF018C020F08B
:1001E00019C021F01AC022F01BC023F01CC024F05B
:1001F00037C03AF037C038F039C03BF04CB012008D
:1002000041C044F042C045F043C046F049C048F008
:1002100049C04AF047C04BF01200476608D04C6A0C
:1002200041C03DF042C03EF043C03FF012004A2EB4
:100230000CD049C04AF04B2E08D047C04BF048665E
:1002400002D04C6AEDD74C80482E48504A5CD8B05A
:10025000E7D744C03DF045C03EF046C03FF0120035
:10026000D3507009D36E9B8C00EE00F0EE50002648
:1002700000B0012AEAA0FAD700EE00F0006602D032
:10028000450E006E016602D0300E016EA6EC0DF038
:100290005CEC0FF00A50AA0A0EE0A6EC0DF00C0E72
:1002A000026E0B0E046EF90E076E050E086E036AE1
:1002B000056A066A096AC26A0F0EC16E070EB46E3D
:1002C000FF0E926E896E936AF00E946E8A6A8B6A44
:1002D000010E396E100E376E050E476E400E496ED8
:1002E0000C0E526E516A506A4F6A0880300E576E7B
:1002F000050E596EC10ED56ED66ACA6ACC6A4B0E0F
:10030000CA6E07C0CBFFCA84F26A9D6AA06A9E6A61
:10031000F06AC00EF16E020E9F6ED08E9D82E00ECE
:10032000F26E82BA20D082B815D0080E1B6E0C0E69
:10033000026E046E036A056A066AF90E076E086AA1
:10034000096A0A6A50EC0FF005EC10F0300E5762A3
:10035000FDD7FF00800E1B6E09804EEC0FF005EC00
:1003600010F082AAFCD7FF0E156E166E176E186E6F
:10037000196E1A6E1B6E1C6EE8EC00F0640E3FECFA
:100380000DF0400E416E426E436EFA0E3FEC0DF0E2
:10039000FA0E3FEC0DF07BEC0DF0640E3FEC0DF02F
:1003A00012C013F011C012F010C011F04EEC0DF09D
:1003B00000503F0B106E116201D0F8D7126201D0CD
:1003C000F5D7136201D0F2D70150070B01092D6E4A
:1003D0004EEC0DF001381F0B0709356E7BEC0DF06C
:1003E00055BE9DEF04F0F950040EFA6E1050040D46
:0403F000F35000D0F6
:10040000F92681EF02F0B0EF02F006EF03F058EFAB
:1004100003F084EF03F098EF03F0B6EF03F0D1EFB1
:1004200003F0E2EF03F00FEF04F027EF04F040EFEA
:1004300004F07DEF04F09DEF04F0A3EF04F0BCEFB7
:1004400004F0E2EF04F0F8EF04F00FEF05F02CEF0A
:1004500005F0E9EF05F0B6EF06F0F5EF06F02CEF4A
:1004600007F075EF07F057EF08F0B5EF09F0DBEF95
:1004700009F047EF0AF0BFEF0AF0E6EF0AF008EFE5
:100480000BF024EF0BF053EF0BF086EF0BF0B6EF11
:100490000BF0D2EF0BF004EF0CF034EF0CF04DEF5B
:1004A0000CF08EEF0CF0C1EF0CF0DDEF0CF010EF64
:1004B0000DF07DEF04F0E9EF05F0F5EF06F0DBEF6E
:1004C00009F0B6EF0BF08EEF0CF004EF0CF084EFB8
:1004D00003F0E2EF03F00FEF05F0B6EF06F075EF73
:1004E00007F024EF0BF0D2EF0BF04DEF0CF098EF8C
:1004F00003F00FEF04F0A3EF04F0B5EF09F0C1EF44
:100500000CF01E0E2D264EEC0DF001501F0B0709AE
:10051000356E0150070B476E030B396EE8EC00F0A7
:100520004EEC0DF000C015F001C016F04EEC0DF0D1
:1005300000C017F001C018F04EEC0DF000C019F02B
:1005400001C01AF04EEC0DF000C01BF001C01CF011
:10055000ACEC0DF035503FEC0DF02D2EDFD720D751
:10056000090E476E030E396EE8EC00F0FF0E156EB3
:10057000166E176E186E196E1A6E1B6E1C6EACEC32
:100580000DF0C80E3FEC0DF0E86AB0EC0DF04EEC4B
:100590000DF001500F0B0109356E0150030B396E40
:1005A000EA6A150EE96E4EEC0DF0070E0014E9260E
:1005B0004EEC0DF0070E01142F6EFE0E306E2F5212
:1005C000D8B404D0304630502F2EFCD7E8EC00F0E1
:1005D000EFCF30F0EF163050EF6201D0E1D7355059
:1005E0003FEC0DF01566DCD71666DAD71766D8D75C
:1005F0001866D6D71966D4D71A66D2D71B66D0D755
:100600001C66CED7C80E3FEC0DF0CAD6090E476E59
:10061000030E396EE8EC00F0640E3FEC0DF04EEC8A
:100620000DF001500F0B0109356E0150030B396EAF
:10063000EA6A150EE96E4EEC0DF0070E0014E9267D
:100640004EEC0DF0070E01142F6E010E306E2F527E
:10065000D8B404D0304630502F2EFCD7E8EC00F050
:10066000EFCF30F0EF123050EF6201D0E1D73550CC
:100670003FEC0DF0FF0E1518DBE1FF0E1618D8E168
:10068000FF0E1718D5E1FF0E1818D2E1FF0E19184A
:10069000CFE1FF0E1A18CCE1FF0E1B18C9E1FF0EC7
:1006A0001C18C6E1ACEC0DF0C80E3FEC0DF078D68E
:1006B0007BEC0DF04EEC0DF001503F0B0F092D6E51
:1006C0004EEC0DF001380F0B0709356EEA6A150E76
:1006D000E96E4EEC0DF0070E0014E9264EEC0DF01D
:1006E000070E01142F6E010E306E2F52D8B404D0B5
:1006F000304630502F2EFCD7EF6E35503FEC0DF0CA
:10070000EF6A2D2EE3D74CD6100E2F6E7BEC0DF03A
:10071000D89035303FEC0DF087EC0DF035503FECC4
:100720000DF0380E2F18D8A4F1D72D2EEDD738D6CE
:100730000150030B476E396E35503FEC0DF0E8EC7D
:1007400000F0FF0E156E166E176E186E196E1A6E8B
:100750001B6E1C6EACEC0DF035503FEC0DF0E8EC70
:1007600000F07BEC0DF02D2EE7D71AD67BEC0DF0C8
:10077000030E2D16070E2F6EEA6A150EE96E010E96
:10078000306E01D030463050EF6E080E3FEC0DF069
:10079000EF6A30AEF7D7E92A2F2EF1D72D2EEAD700
:1007A000FFD5050E306E600E2F6EE8EC00F087EC82
:1007B0000DF035503FEC0DF0302ED5EF03F02D2E1F
:1007C000F0D7EED54EEC0DF001503F0B0F09356E12
:1007D0000150030B396E010B476E4EEC0DF0070E06
:1007E0000114F66E200EF76E0800E8EC00F0F550EC
:1007F000156E166E176E186E196E1A6E1B6E1C6EC5
:10080000030EF66402D0E86A02D0F650010FB0EC95
:100810000DF035503FEC0DF02D2EDFD7C1D5090E70
:10082000476E030E396EE8EC00F07BEC0DF03550AE
:100830003FEC0DF02F6AE8EC00F0ACEC0DF087EC2B
:100840000DF035503FEC0DF02D2EE9D7A9D57BECFE
:100850000DF0010E306E01D03046E8EC00F0305063
:10086000156E166E176E186E196E1A6E1B6E1C6E54
:1008700035503FEC0DF030AEEFD72D2EEAD790D5A6
:10088000060E476E7BEC0DF0800E1B6E35503FEC74
:100890000DF07BEC0DF0800E1C6E35503FEC0DF032
:1008A0007BEC0DF0800E186E35503FEC0DF07BECBC
:1008B0000DF0800E1A6E35503FEC0DF07BEC0DF014
:1008C000800E196E35503FEC0DF02D2ED9D77BECF4
:1008D0000DF0040EB0EC0DF0800E1B6E1C6E186E49
:1008E0001A6E196E640E3FEC0DF0E8EC00F07BEC34
:1008F0000DF03C0E3FEC0DF053D57BEC0DF00150AC
:10090000030B396E010B476E35503FEC0DF035503F
:100910003FEC0DF0E8EC00F0ACEC0DF0380E2F6E73
:10092000E8EC00F087EC0DF035503FEC0DF0600E78
:100930002F62F6D72D2EE1D733D57BEC0DF0C80E04
:100940003FEC0DF02DD57BEC0DF0010E306E01D09B
:100950003046E8EC00F0305015121612171218123B
:1009600019121A121B121C1235503FEC0DF030AE4A
:10097000EFD72D2EE8D714D5060E476E4EEC0DF0AE
:10098000030E0114396EF66E200EF76E0900E8ECC6
:1009900000F0F550156E166E176E186E196E1A6E01
:1009A0001B6E1C6EACEC0DF0C80E3FEC0DF0C80ECB
:1009B0003FEC0DF0E8EC00F07BEC0DF0320E3FEC7C
:1009C0000DF0EED47BEC0DF0060E476E4EEC0DF004
:1009D000030E0114396EE8EC00F02F6A87EC0DF07D
:1009E000ACEC0DF035503FEC0DF02D2EF9D7D8D4EE
:1009F0007BEC0DF0060E476E4EEC0DF0030E01146D
:100A0000396EE8EC00F0080E2F6E87EC0DF0ACECC0
:100A10000DF035503FEC0DF02D2EF9D7C1D4060E58
:100A2000476E4EEC0DF0030E0114396E7BEC0DF0A9
:100A3000E8EC00F02F6A87EC0DF035503FEC0DF03C
:100A4000E8EC00F0080E2F6E87EC0DF035503FEC0F
:100A50000DF02D2EEBD7A4D42D50030B2D6E396A3B
:100A6000476A7BEC0DF0800E1B6E35503FEC0DF0AD
:100A700035503FEC0DF07BEC0DF0400E1B6E200E60
:100A80001C6E35503FEC0DF07BEC0DF0030E156E37
:100A900035503FEC0DF07BEC0DF0600E156E3550CF
:100AA0003FEC0DF07BEC0DF0030E166E35503FEC75
:100AB0000DF07BEC0DF0100E186E100E1A6E355006
:100AC0003FEC0DF07BEC0DF0020E186E020E196E6D
:100AD00035503FEC0DF07BEC0DF0100E1C6E100E3F
:100AE000196E35503FEC0DF07BEC0DF0800E1C6E56
:100AF000800E196E35503FEC0DF07BEC0DF0200EA2
:100B0000186E400E1A6E35503FEC0DF07BEC0DF078
:100B1000020E176E010E1C6E35503FEC0DF07BEC93
:100B20000DF0200E176E400E166E35503FEC0DF096
:100B30007BEC0DF0010E176E010E1B6E35503FEC75
:100B40000DF07BEC0DF0400E176E200E166E35503A
:100B50003FEC0DF07BEC0DF0010E186E020E1B6EDB
:100B600035503FEC0DF07BEC0DF0400E1C6E200E6E
:100B70001B6E35503FEC0DF07BEC0DF0800E186EC7
:100B8000800E1A6E35503FEC0DF07BEC0DF0400EF0
:100B9000186E200E1A6E35503FEC0DF07BEC0DF008
:100BA000010E196E020E1A6E35503FEC0DF07BEC03
:100BB0000DF0600E196E35503FEC0DF07BEC0DF032
:100BC000010E1A6E35503FEC0DF02D2E4AD7D0EFA6
:100BD00001F02D50030B2D6E0150030B396E476A47
:100BE0007BEC0DF0E8EC00F0800E1B1235503FEC72
:100BF0000DF035503FEC0DF0E8EC00F0400E1B120C
:100C0000200E1C1235503FEC0DF0E8EC00F0030E06
:100C1000151235503FEC0DF0E8EC00F0600E1512A7
:100C200035503FEC0DF0E8EC00F0030E1612355095
:100C30003FEC0DF0E8EC00F0100E1812100E1A1236
:100C400035503FEC0DF0E8EC00F0020E1812020EE9
:100C5000191235503FEC0DF0E8EC00F0100E1C12AC
:100C6000100E191235503FEC0DF0E8EC00F0800E3C
:100C70001C12800E191235503FEC0DF0E8EC00F01C
:100C8000200E1812400E1A1235503FEC0DF0E8EC11
:100C900000F0020E1712010E1C1235503FEC0DF041
:100CA000E8EC00F0200E1712400E161235503FEC03
:100CB0000DF0E8EC00F0010E1712010E1B1235507A
:100CC0003FEC0DF0E8EC00F0400E1712200E16126B
:100CD00035503FEC0DF0E8EC00F0010E1812020E5A
:100CE0001B1235503FEC0DF0E8EC00F0400E1C12EA
:100CF000200E1B1235503FEC0DF0E8EC00F0800E9A
:100D00001812800E1A1235503FEC0DF0E8EC00F08E
:100D1000400E1812200E1A1235503FEC0DF0E8EC80
:100D200000F0010E1912020E1A1235503FEC0DF0B0
:100D3000E8EC00F0600E191235503FEC0DF0E8ECD5
:100D400000F0010E1A1235503FEC0DF0ACEC0DF036
:100D5000640E3FEC0DF0E8EC00F07BEC0DF035504C
:100D60003FEC0DF02D2E3CD7D0EF01F00150030BDE
:100D7000396E476A7BEC0DF0E8EC00F0C00E1B12F8
:100D8000200E1C1235503FEC0DF07BEC0DF0E8EC22
:100D900000F0900E1912400E1A1235503FEC0DF073
:100DA0007BEC0DF0E8EC00F0A00E1A12200E1B12E6
:100DB00035503FEC0DF07BEC0DF0E8EC00F0C00E90
:100DC0001812400E1C1235503FEC0DF07BEC0DF06C
:100DD000E8EC00F0900E1C12200E181235503FEC7B
:100DE0000DF02D2EC7D7D0EF01F07BEC0DF00C0EDF
:100DF0001512080E1B1235503FEC0DF07BEC0DF078
:100E0000040E1812040E1712040E1C1235503FEC7B
:100E10000DF07BEC0DF0080E1712080E1812080EDC
:100E2000191235503FEC0DF07BEC0DF0040E191249
:100E3000040E1A12040E1B1235503FEC0DF07BEC21
:100E40000DF00C0E1612080E1A1235503FEC0DF074
:100E50002D2ECBD7D0EF01F07BEC0DF0C80E1B127E
:100E6000200E1C120C0E151235503FEC0DF07BECD1
:100E70000DF0900E1912400E1A12040E1812040EE4
:100E80001712040E1C1235503FEC0DF07BEC0DF0E8
:100E9000A00E1A12200E1B12080E1712080E18129E
:100EA000080E191235503FEC0DF07BEC0DF0C00E22
:100EB0001812400E1C12040E1912040E1A12040EFF
:100EC0001B1235503FEC0DF07BEC0DF0900E1C1218
:100ED000200E18120C0E1612080E1A1235503FEC86
:100EE0000DF02D2EB9D7D0EF01F00150030B396E64
:100EF000476A4EEC0DF001501F0B0709356E030ECB
:100F00002D167BEC0DF0E8EC00F0010E16123550BA
:100F10003FEC0DF0E8EC00F0010E171235503FECFD
:100F20000DF0E8EC00F0010E1A1235503FEC0DF018
:100F3000E8EC00F0010E1B1235503FEC0DF0E8EC30
:100F400000F0020E161235503FEC0DF0E8EC00F008
:100F5000100E1812200E171235503FEC0DF0E8EC71
:100F600000F0400E1712400E191235503FEC0DF0F4
:100F7000E8EC00F0200E1612200E191235503FEC4E
:100F80000DF0E8EC00F0100E1A12400E161235505B
:100F90003FEC0DF0E8EC00F0600E151235503FEC20
:100FA0000DF0E8EC00F0020E1712020E1812355088
:100FB0003FEC0DF0E8EC00F0010E1812010E1912D2
:100FC00035503FEC0DF0E8EC00F0020E1A12020E64
:100FD0001B1235503FEC0DF0E8EC00F0010E1C1236
:100FE000020E191235503FEC0DF0E8EC00F0030E44
:100FF000151235503FEC0DF0E8EC00F0100E1C120D
:10100000200E181235503FEC0DF0E8EC00F0400EC9
:101010001C12400E181235503FEC0DF0E8EC00F0B9
:10102000200E1A12200E1B1235503FEC0DF0E8EC8A
:1010300000F0100E1912400E1A1235503FEC0DF050
:10104000E8EC00F0200E1C12400E1B1235503FEC55
:101050000DF0E8EC00F0800E1C1235503FEC0DF066
:10106000E8EC00F0800E181235503FEC0DF0E8EC83
:1010700000F0800E1A1235503FEC0DF0E8EC00F055
:10108000800E191235503FEC0DF0E8EC00F0800EA8
:101090001B1235503FEC0DF0ACEC0DF0640E3FEC44
:1010A0000DF0E8EC00F02D2E2CD7D0EF01F07BEC0A
:1010B0000DF0800E1B6E400E156E35503FEC0DF09E
:1010C0007BEC0DF0200E1C6E010E156E35503FECC2
:1010D0000DF07BEC0DF0020E156E400E1B6E3550C0
:1010E0003FEC0DF07BEC0DF0200E156E800E1B6EAC
:1010F00035503FEC0DF07BEC0DF0020E166E200E1D
:101100001C6E35503FEC0DF07BEC0DF0100E1A6E9E
:10111000020E156E35503FEC0DF07BEC0DF0020E1B
:10112000196E200E156E35503FEC0DF07BEC0DF076
:10113000100E196E020E166E35503FEC0DF07BEC62
:101140000DF0800E196E100E1A6E35503FEC0DF03A
:101150007BEC0DF0400E1A6E020E196E35503FEC0E
:101160000DF07BEC0DF0010E1C6E100E196E35505B
:101170003FEC0DF07BEC0DF0400E166E800E196EFC
:1011800035503FEC0DF07BEC0DF0010E1B6E400E68
:101190001A6E35503FEC0DF07BEC0DF0200E166E04
:1011A000010E1C6E35503FEC0DF07BEC0DF0020E85
:1011B0001B6E400E166E35503FEC0DF07BEC0DF0C3
:1011C000210E1B6E35503FEC0DF07BEC0DF0800EC8
:1011D0001A6E200E166E35503FEC0DF07BEC0DF0C4
:1011E000200E1A6E020E1B6E35503FEC0DF07BEC9C
:1011F0000DF0020E1A6E200E1B6E35503FEC0DF0F6
:101200007BEC0DF0200E196E800E1A6E35503FECFF
:101210000DF07BEC0DF0210E1A6E35503FEC0DF009
:101220007BEC0DF0400E196E020E1A6E35503FEC3D
:101230000DF07BEC0DF0210E196E35503FEC0DF0EA
:101240007BEC0DF0400E186E010E1A6E35503FEC1F
:101250000DF07BEC0DF0800E186E400E196E3550BF
:101260003FEC0DF07BEC0DF0400E1C6E010E196E84
:1012700035503FEC0DF07BEC0DF0410E186E355003
:101280003FEC0DF07BEC0DF0400E176E800E186EEB
:1012900035503FEC0DF07BEC0DF0010E176E400E5B
:1012A0001C6E35503FEC0DF07BEC0DF0200E176EF0
:1012B000010E186E35503FEC0DF07BEC0DF0420E38
:1012C000176E35503FEC0DF07BEC0DF0200E186ED4
:1012D000010E176E35503FEC0DF07BEC0DF0800EDB
:1012E0001C6E200E176E35503FEC0DF07BEC0DF0B0
:1012F000100E1C6E020E176E35503FEC0DF07BEC9D
:101300000DF0220E186E35503FEC0DF07BEC0DF019
:10131000100E186E800E1C6E35503FEC0DF07BECFD
:101320000DF0010E166E100E1C6E35503FEC0DF0D8
:101330007BEC0DF0400E156E020E186E35503FEC32
:101340000DF07BEC0DF0010E156E100E186E355081
:101350003FEC0DF07BEC0DF0400E1B6E010E166E97
:1013600035503FEC0DF0D0EF01F04EEC0DF0015098
:10137000070B476E030B396EE8EC00F07BEC0DF0C9
:10138000050E306E35503FEC0DF0580E2F6EE8EC28
:1013900000F087EC0DF0100E2F5E35503FEC0DF095
:1013A000302EF5D7ACEC0DF035503FEC0DF02D2E76
:1013B000E3D7D0EF01F07BEC0DF0800E1B6E800EBA
:1013C000196E800E1A6E800E186E800E1C6E3550CF
:1013D0003FEC0DF07BEC0DF0700E1C6E600E1A6E83
:1013E00035503FEC0DF07BEC0DF0020E156E010E4A
:1013F0001C6E020E1A6E030E186E35503FEC0DF087
:101400007BEC0DF0200E156E400E166E200E196E40
:10141000400E176E100E186E35503FEC0DF07BEC41
:101420000DF0030E166E010E1B6E010E1A6E010EEC
:10143000176E35503FEC0DF07BEC0DF0100E1A6E70
:10144000200E166E400E196E200E176E400E156E91
:1014500035503FEC0DF07BEC0DF0030E196E020ED3
:101460001B6E020E176E010E156E35503FEC0DF01F
:101470007BEC0DF0100E196E600E1B6E600E186E78
:1014800035503FEC0DF02D2E96D7D0EF01F04EECFD
:101490000DF00150070B396E476AE8EC00F07BEC69
:1014A0000DF00C0E156E35503FEC0DF035503FEC45
:1014B0000DF0E8EC00F07BEC0DF0030E166E3550ED
:1014C0003FEC0DF0E8EC00F07BEC0DF0100E186E28
:1014D000100E1A6E35503FEC0DF0E8EC00F07BEC8E
:1014E0000DF0020E186E020E196E35503FEC0DF025
:1014F000E8EC00F07BEC0DF0100E1C6E100E196E77
:1015000035503FEC0DF0E8EC00F07BEC0DF0800E78
:101510001C6E800E196E35503FEC0DF035503FECCF
:101520000DF0E8EC00F07BEC0DF0100E1C6E100ED0
:10153000196E35503FEC0DF0E8EC00F07BEC0DF04F
:10154000020E186E020E196E35503FEC0DF0E8ECED
:1015500000F07BEC0DF0100E186E100E1A6E355068
:101560003FEC0DF0E8EC00F07BEC0DF0030E166E96
:1015700035503FEC0DF02D2E90D7D0EF01F07BECE5
:101580000DF0100E156E35503FEC0DF07BEC0DF0AC
:10159000100E1B6E35503FEC0DF07BEC0DF0100E75
:1015A000166E35503FEC0DF07BEC0DF0800E156E95
:1015B00035503FEC0DF07BEC0DF0100E176E3550F2
:1015C0003FEC0DF02D2EDBD7D0EF01F07BEC0DF0D2
:1015D000476A030EB0EC0DF0E86A2F6E87EC0DF051
:1015E000800E1B121C1218121A12191235503FECE1
:1015F0000DF035503FEC0DF01B9E1C9E189E1A9E60
:10160000199E35503FEC0DF02D2EEAD7D0EF01F0AA
:101610007BEC0DF0040E2E6E0F0E2F6E060E306E4C
:10162000800E1B121C1218121A1219122F503FECA6
:101630000DF07BEC0DF030503FEC0DF02E2EF0D77E
:101640002D2EE6D7D0EF01F04EEC0DF00150070B38
:10165000396E260EF76E2E6A00C02FF00F0E35166B
:101660002FB20ED0E8EC00F02E5030EC13F03550D5
:101670003FEC0DF02E2A0B0E2E64F2D72FB00ED0B9
:101680000B0E2E6EE8EC00F02E5030EC13F03550BF
:101690003FEC0DF02E06FF0E2E62F4D72E6A2D2E93
:1016A000DFD7D0EF01F04EEC0DF00150070B396E93
:1016B000476E030EB0EC0DF0230EF76E2E6A00C0DD
:1016C0002FF00F0E35162FB20ED0E8EC00F02E5092
:1016D00030EC13F035503FEC0DF02E2A050E2E6441
:1016E000F2D72FB00ED0050E2E6EE8EC00F02E5083
:1016F00030EC13F035503FEC0DF02E06FF0E2E624D
:10170000F4D72E6A2D2EDFD7D0EF01F04EEC0DF07E
:101710000150070B396E476E220EF76E2E6A00C01D
:101720002FF00F0E35162FB20ED0E8EC00F02E5031
:1017300030EC13F035503FEC0DF02E2A0B0E2E64DA
:10174000F2D72FB00ED00B0E2E6EE8EC00F02E501C
:1017500030EC13F035503FEC0DF02E06FF0E2E62EC
:10176000F4D72E6A2D2EDFD7D0EF01F04EEC0DF01E
:101770000150070B396E476E070E3516270EF76EB0
:101780002E6AE8EC00F02E5030EC13F035503FECB0
:101790000DF02E2A330E2E64F4D7640E3FEC0DF0BC
:1017A000D0EF01F0030E2D124EEC0DF00150010BA5
:1017B000396E476EACEC0DF0290EF76E2E6A00C044
:1017C0002FF02FB20ED0E8EC00F02E5030EC13F0DA
:1017D00035503FEC0DF02E2A040E2E64F2D72FB0B8
:1017E0000ED0040E2E6EE8EC00F02E5030EC13F00C
:1017F00035503FEC0DF02E06FF0E2E62F4D72E6A08
:101800002D2EDFD7D0EF01F0030E2D124EEC0DF090
:101810000150010B396E476E2A0EF76E2E6A00C01A
:101820002FF02FB20ED0E8EC00F02E5030EC13F079
:1018300035503FEC0DF02E2A040E2E64F2D72FB057
:101840000ED0040E2E6EE8EC00F02E5030EC13F0AB
:1018500035503FEC0DF02E06FF0E2E62F4D72E6AA7
:101860002D2EDFD7D0EF01F0050E476E030E396E37
:10187000030E2D12E8EC00F0290EF76E280EF66E1E
:1018800033EC13F0E8EC00F0ACEC0DF0640E3FEC40
:101890000DF02D2EF7D7D0EF01F0010E396E040EAA
:1018A0002D26210EF76E09D0E8EC00F0680EF66EDA
:1018B00033EC13F0640E3FEC0DF0E8EC00F0700E2A
:1018C000F66E33EC13F0140E3FEC0DF0E8EC00F084
:1018D000780EF66E33EC13F0140E3FEC0DF0E8ECDE
:1018E00000F0800EF66E33EC13F0640E3FEC0DF05A
:1018F000E8EC00F0780EF66E33EC13F0140E3FECCB
:101900000DF0E8EC00F0700EF66E33EC13F0140EF0
:101910003FEC0DF02D2EC8D7D0EF01F0030E2D12A5
:101920004EEC0DF00150010B396E476E0B0EB0EC12
:101930000DF02B0EF76E2E6A00C02FF02FB20ED0D6
:10194000E8EC00F02E5030EC13F035503FEC0DF089
:101950002E2A040E2E64F2D72FB00ED0040E2E6E57
:10196000E8EC00F02E5030EC13F035503FEC0DF069
:101970002E06FF0E2E62F4D72E6A2D2EDFD7D0EF63
:1019800001F0010E396E030E2D122B0EF76EE8ECEE
:1019900000F0280EF66E33EC13F03C0E3FEC0DF029
:1019A000E8EC00F0300EF66E33EC13F0280E3FEC4E
:1019B0000DF02D2EECD7D0EF01F0030E2D124EECD2
:1019C0000DF00150010B396E476E0A0EB0EC0DF0B0
:1019D0002C0EF76E2E6A00C02FF02FB20ED0E8EC5E
:1019E00000F02E5030EC13F035503FEC0DF02E2A65
:1019F000040E2E64F2D72FB00ED0040E2E6EE8EC3B
:101A000000F02E5030EC13F035503FEC0DF02E0668
:101A1000FF0E2E62F4D72E6A2D2EDFD7D0EF01F005
:101A2000030E2D124EEC0DF00150010B396E2D0EF0
:101A3000F76E2E6A00C02FF02FB20ED0E8EC00F047
:101A40002E5030EC13F035503FEC0DF02E2A040EE2
:101A50002E64F2D72FB00ED0090E2E6EE8EC00F0F7
:101A60002E5030EC13F035503FEC0DF02E06040EE6
:101A70002E62F4D72E6A2D2EDFD7D0EF01F0346E10
:101A800057A8DBEC0DF057BA06D0557E57AAFED703
:101A90000600D0EF01F03466F3D71200016603D0E0
:101AA000300ED624016E006602D0450E006E013461
:101AB0000118E836013A0038E8460118013A010BEE
:101AC0000036001A01361200016602D0350E016E92
:101AD000006602D0490E006E0034003400B8010ADE
:101AE00000BA010A00B6010A006E1D0ED890013638
:101AF000D8B0011A1200156A166A176A186A196AAC
:101B00001A6A1B6A1C6A4C6AE86A2AD012002FC043
:101B1000F6FF210EF76E0900F5CF15F00900F5CF9D
:101B200016F00900F5CF17F00900F5CF18F00900FD
:101B3000F5CF19F00900F5CF1AF00900F5CF1BF029
:101B40000900F5CF1CF0080E2F26120000EE02F05F
:101B5000EE6AE9AEFDD712004EEC0DF000501F0BFF
:101B60004CB01200040DF3CFF6FF2E0EF76E0900F5
:101B7000F5CF41F00900F5CF42F00900F5CF43F071
:101B800012004F2A630E4F64010C4F6A562A502AE6
:101B90003B0E5064010C506A512A3B0E5164000CFC
:101BA000516A522A0C0E526201D008705264000C25
:101BB000010E526E000C55845590476A396AE86AE6
:101BC000B0EC0DF0566A030E566028D07BEC0DF099
:101BD000E8EC00F057A8F7D7520490EC0EF008B0EC
:101BE000238E23C01BF057BA04D0D0EC0DF08DEC3F
:101BF0000EF057B8F1D77BEC0DF08AEC0EF0515097
:101C0000AEEC0EF057BA04D020EC0FF08DEC0EF0D5
:101C100057A877D0780E5664F2D773D055827BECF4
:101C20000DF0010EB0EC0DF08AEC0EF0020490EC19
:101C30000EF008B2238E23C01BF057BA05D028EC53
:101C40000FF08DEC0EF0558057B8F0D77BEC0DF00F
:101C5000010EB0EC0DF08AEC0EF00350AEEC0EF07D
:101C600057BA04D032EC0FF08DEC0EF057A804D028
:101C7000780E5664F2D745D055827BEC0DF0020EFB
:101C8000B0EC0DF08AEC0EF0040490EC0EF008B409
:101C9000238E23C01BF057BA04D038EC0FF08DEC24
:101CA0000EF057B8F1D77BEC0DF0020EB0EC0DF052
:101CB0008AEC0EF00550AEEC0EF057BA05D042ECAF
:101CC0000FF08DEC0EF0558057A804D0780E5664B6
:101CD000F1D717D055827BEC0DF0030EB0EC0DF070
:101CE0008AEC0EF0F5EC0EF057BA05D048EC0FF088
:101CF0008DEC0EF0558057A804D0780E5664F2D7BC
:101D000000D08AEC0EF0559255B04EEC0FF0559085
:101D1000559E120057A8FED7120057AAFED71200F0
:101D2000080DF3CFF6FF220EF76E0900F5CF15F080
:101D30000900F5CF16F00900F5CF17F00900F5CF2F
:101D400018F00900F5CF19F00900F5CF1AF00900D5
:101D5000F5CF23F00900F5CF1CF0120017EC0FF0BF
:101D60005350080DF3CFF6FF230EF76E0900F5CFA1
:101D70001DF00900F5CF1EF00900F5CF1FF0090096
:101D8000F5CF20F00900F5CF21F00900F5CF22F0C2
:101D90000900F5CF23F00900F5CF24F05450080DC9
:101DA000F3CFF6FF240EF76E0900F5501D10156EE7
:101DB0000900F5501E10166E0900F5501F10176E21
:101DC0000900F5502010186E0900F5502110196E09
:101DD0000900F55022101A6E0900F55023101B6EF1
:101DE0000900F55024101C6E12000650080DF3CFA8
:101DF000F6FF250EF76E0900F5CFCBFFF5CF07F004
:101E0000156A0900F5CF16F00900F5CF17F00900A3
:101E1000F5CF18F00900F5CF19F00900F5CF1AF049
:101E20000900F5CF1BF00900F5CF1CF01200546E2D
:101E3000536A0A0E545CD8A01200546E532AF9D784
:101E40004F6A506A512A3B0E51641200516A1200C7
:101E5000022A0C0E026201D0087202641200010E06
:101E6000026E1200032A3B0E03641200036A120082
:101E7000042A0C0E046201D0087404641200010EDE
:101E8000046E1200052A3B0E05641200056A12005A
:101E9000062A0E0E06641200066A1200AA0E0A6EC8
:101EA0004D6A090E4E6E00EE02F0EE5069EC0FF036
:101EB0004D2A4E2EFAD712004D6A090E4E6E00EED4
:101EC00002F04D507AEC0FF0EE6E4D2A4E2EF9D7FF
:101ED0001200A6B2FED7A86E4DC0A9FFA69EA69C72
:101EE000A684F29E550EA76EAA0EA76EA682F28E4B
:101EF000A6941200A96EA69EA69CA680A8501200C9
:10200000030CF0FF0FF3FC00FC00230E2E6EB90E44
:102010002F6E090E306E2E2EFED72F2EFCD7302EAF
:04202000FAD71200D9
:102100009C1C1C0C0C0C1C04636363F3F3F3E3F1E1
:10211000632F45C561A3E3600C632B32BAF32391AF
:10212000634345C5D751C561632F2B3228A3E3B064
:102130000C4363F3D75105D10003010000010100F6
:102140006063611060110100636363136313030133
:102150006363637373736371636363F3F3F3E3F153
:10216000630300000000C020004200009250010103
:102170000020000020A32300000041C141010040D5
:08218000000123320000009071
:1022000000000000800000000000000090000000BE
:10221000000000009200000000000000921000008A
:102220000002000092100000040200009210000062
:102230000C020000921000000C030000921000003D
:102240000C030010921000000C030012921000000A
:102250000C030012921000100C0300129210009058
:1023000000000000000000001000000000000000BD
:1023100010001000000000009000100000000000FD
:10232000901010000000000090101000000010003D
:10240000000000000000000000000000008000004C
:102410000000000000A000000000000000A200007A
:102420000000000020A200000000000020A3000027
:102430000000000060A300000000000061A3000095
:102440000000004061A30000000000C061A3000084
:10250000F900000000010000F800000008010000D0
:10251000F700080008010000F600090008010000AB
:10252000F500290008010000F4002B00080100005C
:10253000F3002B2008010000F2002B20080100808E
:10254000FA00000004010000FB0000000401040088
:10255000FC00000004010500FD400000040105002E
:10256000FE40000004010501FF4000000441050198
:08257000FF4000008441050159
:10260000000000008000000000000000100000003A
:1026100000000000020000000000000000100000A8
:1026200000020000000000000400000000000000A4
:102630000800000000000000000100000000000091
:102640000000001000000000000000020000000078
:1026500000000000000000100000000000000080EA
:10266000080DF3CFF6FF0900F5CF15F00900F5CFFF
:1026700016F00900F5CF17F00900F5CF18F00900A2
:10268000F5CF19F00900F5CF1AF00900F5CF1BF0CE
:082690000900F5CF1CF0120057
:102700000000000000000000000000000000008049
:102710000000000000000090000000020000009097
:102720000000001200000090000100120000009064
:1027300008010012000000900C010012000000903F
:102740000C030012000000900C0300120010009017
:102750000C030012021000900C03001212100090E3
:102760000C030012921000900C0300129250009083
:102770000C030012925000910C43001292500091F1
:102780000C430012925001910C430012925005919B
:102790000C430012965005910C430012965105917E
:1027A0000C430012D65105910C430012D6510591ED
:1027B0000C430012D75105910C430052D75105919B
:1027C0000C4300D2D75105910C4300D2D75105D10B
:1027D0000C4300D3D75105D10C4340D3D75105D179
:1027E0000C4341D3D75105D10C4345D3D75105D123
:1027F0000C4345D7D75105D14C4345D7D75105D1C7
:102800004D4345D7D75105D14D4345D7D75145D134
:102810004D4345D7D751C5D14D4345D7D751C5F1C4
:102820004F4345D7D751C5F16F4345D7D751C5F170
:102830006F4745D7D751C5F16F4F45D7D751C5F130
:102840006F6F45D7D751C5F16F6F45D7D751C7F1D6
:102850006F6F45D7D751E7F16F6F45D7D7D1E7F104
:102860006F6F45D7D7F1E7F16F6F45D7D7F3E7F132
:102870006F6F45D7F7F3E7F16F6F45D7FFF3E7F1D8
:102880006F6F4DD7FFF3E7F16F6F6DD7FFF3E7F190
:102890006F6F6FD7FFF3E7F16F6F6FF7FFF3E7F13C
:102900009C1018080C041C00901C1C0C08081004D7
:102910009C10140404041C049C1C180808081800CB
:10292000901C1404040C1404030303838383838125
:102A00000C03001292100090004000C0C541050167
:102A1000410145850000C040222E00000080A32017
:082A200000002B2028A3008018
:102B000022020000921090200070000080C023017B
:102B1000800000C061A30000000073A1000000C09D
:102B2000510100120000C09000402B208C41058113
:082B3000000000C061A30000D9
:102C00000C03000000000000000E000000000100A6
:102C10000000000004010500000009000801000098
:082C20000001050400000000A2
:102D0000410100000000C00000020000921000001D
:102D10000020000000802300000000C041010000EE
:102D200000002320000000800040000080400101DE
:102D30000000000020A300000000418100000040CE
:102D4000000100120000009022020000000080201C
:102E00000000000040000000004000000000400002
:102E10004040400020000000002000000000200092
:102E2000202020000A000000000A000000000A0024
:102E30000A0A0A00400040004040000000404000F4
:102E400040280000190D4000330D4000400D3300B4
:102E5000400D1900401A0D0040331A0033400D0098
:102E60001A400D000D401A000D4033000D33400094
:102E70000D1A4000000E3A002B003A003A000E00F6
:102E80000E3A0000684369727473616D2073745365
:102E9000726176202E3020336F43797069726867D3
:102EA00020742E446854726F6570322030302036A2
:102EB00077772E776E7573756175656C656C746365
:102EC0006F72696E7363632E2E6F6B75702F6F72E6
:0E2ED000656A74632F7374737261702E70687C
:020000040030CA
:0300010008121EC4
:020005008081F8
:060008000FC00FE00F40E5
:00000001FF
